:10000000000003308A00072B8030A100FE304A2117
:1000100001304A217530A80030308C29A101A11788
:10002000B600FE304A2136084A29A501AF00B001CA
:10003000A01125080319A0150530A4002730AC0035
:1000400010302E200330AC00E8302E20AC0164309C
:100050002E20AC010A302E202F083528AB003008A6
:10006000A8002F08A70015222708A700A40303193A
:10007000A011250803193F28240203184628270841
:10008000031DA011A0194628303E4A290800C800C7
:10009000B91F4C282D304A21BB0F5328BA0F5328C3
:1000A000B90A0319B90AC001C101C201C301B917D4
:1000B0006A30B8070310B90CBA0CBB0CC30CC20CE5
:1000C000C10CC00CB80F5A283B083802BB07B80255
:1000D0003A083902BA07B902A501A6202E304A21F2
:1000E000C9010310400DBB00410DBA00420DB9001B
:1000F000430DB800C90D0310BB0DBA0DB90DB80DF5
:10010000C90D4008BB0741080318410FBA07420850
:100110000318420FB90743080318430FB807031821
:10012000C90F0310BB0DBA0DB90DB80DC90D4908A3
:10013000303E4A213B08C0003A08C1003908C200DD
:100140003808C300C80B70280310312AA0112508F5
:10015000031DAD28A0150A30A5003B08AA003A08E7
:10016000A9003908A8003808A700A401B201B1010C
:10017000B0010A30AF009B21A40A24082502031D08
:10018000B6282F08031DA011A01DC828250BCB28B9
:100190002F08303E4A21A50BAD28312AB400861124
:1001A00006118316861106110F3086058312340856
:1001B000A018F8283E30A80080308C213330B300DE
:1001C0000C211330A80088308C210C2164308B2145
:1001D0000C2164308B212230B3000C212830F72011
:1001E0000C30F7200630F720A0143408F82820142B
:1001F000B300201C06290611033C031C0B290B210C
:100200000730A800D0308C21031408002014FE3CD5
:1002100003191B290615201C201086150F30860592
:100220003308F039860400008611B30E0000201850
:100230000C2932308B213408312A981818121816DC
:100240002308A7002608A800AB01AC01272928290C
:1002500000008C1A4229FF30AB07031CAC07031CBB
:10026000A707031CA807031C312A2B0F26292C0FD4
:100270002729FA30AB00AC01282998181812181653
:100280008C1E40291A080314312A0C1E4529990096
:100290000314312AA11BCE28211945290800A400E6
:1002A000A201240803178D000313250803178F00EC
:1002B00062210319312A4A21A40A0319A50AA20FAF
:1002C0005129312A831603178C170C1400000000E3
:1002D00083120C08312AB300B30DB30D330D383936
:1002E000C1389F0032308B211F151F1975291E0838
:1002F000B90083161E088312B800312AAC01AB0086
:10030000FF30AB07031CAC07031C312A0330A800E5
:10031000E6308C218029A801FC3EA700A809031C17
:100320009729FF300000A70703189229A7070000AC
:10033000A80F912908002A0832068039B400AA1FA4
:10034000AC29A709A809A909AA09A70A0319A80A93
:100350000319A90A0319AA0AB21FB929AF09B009DA
:10036000B109B209AF0A0319B00A0319B10A031996
:10037000B20AAB01AC01AD01AE01BC01BD01BE01D1
:10038000BF013208310430042F040319F72920304B
:10039000B3000310A70DA80DA90DAA0DBC0DBD0D2E
:1003A000BE0DBF0D32083F02031DE02931083E0299
:1003B000031DE02930083D02031DE0292F083C02FF
:1003C000031CF1292F08BC023008031C300FBD02AA
:1003D0003108031C310FBE023208031C320FBF026A
:1003E0000314AB0DAC0DAD0DAE0DB30BC929B41F8D
:1003F000042AAB09AC09AD09AE09AB0A0319AC0A72
:100400000319AD0A0319AE0A3C08AF003D08B0005D
:100410003E08B1003F08B2002B08A7002C08A80036
:100420002D08A9002E08AA00312AB001AF01103012
:10043000B300280DAF0DB00D2B08AF022C08031C24
:100440002C0FB00203182B2A2B08AF072C08031817
:100450002C0FB0070310A70DA80DB30B192A2708FE
:10046000080083138312031308004108BE004506E9
:10047000CC00C40803199F2AC0080319A22A440803
:10048000C0027F300318482AC007031CA12A4B2A48
:10049000C0070318A42A4308BC004208BD00BE17C9
:1004A000C5171830CB00C301C201C101592A031876
:1004B000652A47083C024608031C460F3D024508D2
:1004C000031C450F3E02031C702A4708BC02460865
:1004D000031C460FBD024508031C450FBE02031452
:1004E000C30DC20DC10DBC0DBD0DBE0DCB0B572AEA
:1004F000C11B822AC0080319A12ACC0CC003CB0A55
:10050000CC0D572A4A1F9E2A0318922A4708BC027C
:100510004608031C460FBD024508031C450FBE02DA
:10052000031C9E2AC30F9E2AC20F9E2AC10F9E2A19
:10053000C10CC20CC30CC00A0319A42AAB2ACA15E9
:10054000A52A4A15C001A72ACA14FF30C000C3015A
:10055000C2018030C100CC1BAE2AC113312AC201B6
:10056000C3019630CB00CC13C31FC22AC309C209F2
:10057000C109C009C00FC12AC10FC12AC20A03198B
:10058000C30ACC17C3080319DD2A4A1FD42AC31F84
:10059000D42AC10FD42AC20FD42AC30FD42A0314D9
:1005A000C30CC20CC10CCB0A0830CB074108C000F9
:1005B0004208C1004308C200F22AC208031DF22A01
:1005C0000830CB024108031DEE2A0830CB02400858
:1005D000031DED2A4308CB00FC2AC001C2004008DD
:1005E000C100C001C21BFA2A0310C00DC10DC20D0B
:1005F000CB03F22ACC1FC2134008C3004B08C00033
:100600004208CB004108C2004B08C100312A8301D7
:10061000831681309900243098008312903098001E
:100620004030CA00A001073083169C009F00803034
:100630008700813099000730850080309F0081302D
:1006400083129F008030A1008A010E200330A50094
:10065000D8308A014F210730AC00D0308A017F2189
:100660008A0104208A110A12352BD101D0010330EE
:10067000A600E830A3008A011D218A110A12031C7A
:10068000572BD0008A011D218A110A12031C572BF7
:10069000D1008030A100C0308A010E20A501510890
:1006A000B0005008AF008A0118208A01352B50088D
:1006B000673A51048A110A12031D652BCF0A8A1169
:1006C0000A12672BC8308A017E218A01352B00303F
:1006D0008A016B21CD003908CE0020308A014521E6
:1006E0008A0145210430A1004F088A0115202E30CF
:1006F0008A01452120308A0145219A30C70099306E
:10070000C6004C30C5008630C4004E08C1004D08FC
:10071000C0008A01AF228A0135224308BB0042088B
:10072000BA004108B9004008B80003308A014720E8
:100730008030A1008A010E2020308A01CE208A015B
:10074000CE204F088A0115202E308A01CE2020307D
:100750008A01CE209A30C7009930C6004C30C500BF
:100760008630C4004E08C1004D08C0008A01AF2287
:100770008A0135224308BB004208BA004108B9008B
:100780004008B80003308A0147208030A100C03003
:100790008A010E20A5015108B0005008AF008A015F
:1007A0001820C8308A017E218A01352B8A01D62B78
:0E07B000500052004900560045005400000061
:02400E00323F3F
:00000001FF
